:020000040000FA
:020000007D2859
:0800080009009801831603139F
:1000100098010C30990024309800C0308B008C1669
:10002000831203138030980008004130322054308E
:1000300032202B30322049303220503032205230A2
:1000400032203D30322031303220393032203230CF
:10005000322030303220303032200D3032200A3021
:10006000322008000C1E3228990008000D30322082
:100070000A303220080041303220543032202B30F8
:100080003220433032204D30322053303220533032
:1000900032203D30322008003B20313032202C30DD
:1000A0003220362008003B20323032202C303220E3
:1000B000362008003B20333032202C3032203620CE
:1000C00008004130322054303220443032203E305B
:1000D0003220533032204D303220313032203B300C
:1000E00032200D303220080041303220543032208E
:1000F000483032200D30322008008B1383128501E6
:1001000007309F0000308316850083128601FB3084
:10011000831686008312C901861EB02A061E522A43
:10012000831679309B001C14831203101A182A2995
:100130009A18DE28A92883120512442244220511A8
:100140008511C910003083169A0079309B00A022D7
:1001500036228312061E522A861EB02A6121C91C2D
:10016000A928B22883120516C910C3013030C30074
:1001700085153622851144226400851544226121AB
:10018000C9189B28C30BBA28051205206400152046
:10019000023083169A0079309B00A0228312C91086
:1001A000851536228511061FD9286121C91CD3283F
:1001B0009B2805108510851544220511831285158D
:1001C0006400FF306200C910061BEA286121C918CB
:1001D0009B28E028C2011B30C20005168515442269
:1001E0006400851144226121C9189B28C20BED28A7
:1001F00005124C206400FF3062000130BD0005157F
:100200008511EC21C91C05299B288515EC21C91CE9
:100210000A299B28BC0BFF28BD0BFF280511061BD4
:10022000122924295A2085150515362236228511D2
:1002300005116121C91C1D299B2836223622362230
:100240003622061B13292429013083169A0079309F
:100250009B00A02283126400FF3062008515051107
:10026000061F37293329EC21C91C37299B28851102
:10027000061F3F293B29EC21C91C2A299B28532012
:100280006400FF306200061BEA28EC21C91C4D29DE
:10029000C91C4D29C91C4D299B2885116400FF30BC
:1002A0006200061BEA28EC21C91C57299B28EC2177
:1002B000C91C5B299B28EC21C91C5F299B2885153B
:1002C000402932220B222C22FD2132222022061C20
:1002D00076291922061C6D2976290B22061C7629FF
:1002E00078219721CC22491D7629BA212C22080099
:1002F0003330B6000830BA002C22361C80298229FF
:1003000019229129000000000000000000003222A4
:1003100019229229000000000000000000000000E7
:100320007C293222B60CBA0B8A2919220800031044
:10033000203084000830BA0083169B018312A62166
:1003400035088000840ABA0B9F2908000830BB00DA
:100350002C22000000000000000032222022061C97
:10036000B329B517B429B513B50C1922BB0BA829AD
:10037000B50D0800C801C9290830C80778304802FF
:10038000031DC929C9102C220B220515362205117F
:10039000080020308400480883169B008312083030
:1003A000BA0083161C148312031083161A088312D2
:1003B0000002031DBC29840A83169B0A8312BA0B10
:1003C000D1290030A000A100A200A300A400A50034
:1003D000A600A700C91408006400FF306200B00145
:1003E000B101A030B200B00BF629FA296121C91C75
:1003F000FA290800B20BF32908000630B100B0005A
:10040000B00B002AB10BFF290730B100B000B00BD0
:10041000072AB10B062A0430B100B000B00B0E2A37
:10042000B10B0D2A0530B100B000B00B152AB10B8D
:10043000142A0430B100B000B00B1C2AB10B1B2AE7
:1004400000000000000000000000000000000000AC
:100450006400FF3062000800061083160610831245
:10046000061008008316061483120800B001B101BB
:100470000530B200B00B3A2AB10B3A2A6400FF30C3
:100480006200B20B3A2A0800B001B1010130B2009B
:10049000B00B482A6400FF306200B10B482AB20B4F
:1004A000482A0800BC01BD01061E522A572ABD0B6E
:1004B000602ABC0B602A0515442205118511A92864
:1004C00085154911322219222C22FD2132222022A7
:1004D000061C572A1922061C6E2A572A0B22061CB4
:1004E000572A78219721CC22491D572A772A83162B
:1004F00078309B001C141A02031D7F2A9A01831670
:100500001A089B0083120830BA00203084000008CB
:1005100083169A00A0228312840A83169B0A8312F0
:10052000BA0B872A83161B089A0078309B00831227
:10053000A022051544220511851144228515522A51
:1005400083161C151C108B1355309D00AA309D007E
:100550009C141C1183128C1FAB2A8C13831208006D
:100560008312003083169B0008309A008312783083
:10057000BA00A02283169B0A8312BA0BB92A05156A
:1005800085154422051185113622783083169B008B
:1005900000309A00A022522ABE0149112008C10051
:1005A000EB222108C100EB222208C100EB22230824
:1005B000C100EB222408C100EB222508C100EB2278
:1005C0002608C100EB222708C100EB2200303E02C2
:1005D0000319491508000830C00041083E06BF0055
:1005E0003F0C3E080318183ABF003F0CBE00031032
:0A05F000C10C4108C00BEE2A080000
:02400E000D3F64
:00000001FF
